:0200000480007A
:100000006F008004732F2034930F80006308FF0378
:10001000930F90006304FF03930FB0006300FF038E
:10002000130F000063040F0067000F00732F2034CC
:1000300063540F006F00400093E19153171F0000BD
:1000400023223FFC6FF09FFF732540F163100500F2
:10005000970200009382020173905230735000188F
:10006000970200009382020273905230B702008020
:100070009382F2FF7390023B9302F0017390023A75
:1000800097020000938282017390523073502030A7
:1000900073503030735040309301000097020000DD
:1000A000938282F673905230130510001315F501F8
:1000B000634C05000F00F00F930110009308D0056A
:1000C000130500007300000093020000638E02001D
:1000D00073905210B7B20000938292107390223046
:1000E00073232030E39A62F47350003097020000CB
:1000F0009382420173901234732540F173002030D3
:10010000B70001FF938000F037110F0F1301F1F0DA
:1001100033F72000B71E000F938E0EF093012000DE
:10012000631CD749B710F00F938000FF37F1F0F050
:100130001301010F33F72000B70EF000938E0E0F5E
:1001400093013000631AD747B700FF009380F00F88
:1001500037110F0F1301F1F033F72000B70E0F0026
:10016000938EFE00930140006318D745B7F00FF05F
:100170009380F00037F1F0F01301010F33F7200006
:10018000B7FE00F0930150006318D743B70001FF9A
:10019000938000F037110F0F1301F1F0B3F020003E
:1001A000B71E000F938E0EF0930160006396D0414E
:1001B000B710F00F938000FF37F1F0F01301010F3B
:1001C00033F12000B70EF000938E0E0F93017000F4
:1001D0006314D13FB70001FF938000F0B3F010002B
:1001E000B70E01FF938E0EF0930180006396D03D11
:1001F00013020000B70001FF938000F037110F0FCA
:100200001301F1F033F7200013030700130212006B
:1002100093022000E31052FEB71E000F938E0EF0E3
:1002200093019000631AD33913020000B710F00F46
:10023000938000FF37F1F0F01301010F33F7200036
:1002400013000000130307001302120093022000A2
:10025000E31E52FCB70EF000938E0E0F9301A00028
:10026000631CD33513020000B700FF009380F00F2A
:1002700037110F0F1301F1F033F7200013000000C6
:100280001300000013030700130212009302200062
:10029000E31C52FCB70E0F00938EFE009301B000DA
:1002A000631CD33113020000B70001FF938000F0FC
:1002B00037110F0F1301F1F033F720001302120072
:1002C00093022000E31252FEB71E000F938E0EF031
:1002D0009301C0006312D72F13020000B710F00F74
:1002E000938000FF37F1F0F01301010F13000000BD
:1002F00033F720001302120093022000E31052FE95
:10030000B70EF000938E0E0F9301D0006316D72B1B
:1003100013020000B700FF009380F00F37110F0F9A
:100320001301F1F0130000001300000033F7200068
:100330001302120093022000E31E52FCB70E0F00BE
:10034000938EFE009301E0006318D727130200008C
:10035000B70001FF938000F01300000037110F0F6A
:100360001301F1F033F72000130212009302200072
:10037000E31052FEB71E000F938E0EF09301F000B3
:10038000631CD72313020000B710F00F938000FF07
:100390001300000037F1F0F01301010F130000000B
:1003A00033F720001302120093022000E31E52FCD8
:1003B000B70EF000938E0E0F93010001631ED71F3E
:1003C00013020000B700FF009380F00F130000003D
:1003D0001300000037110F0F1301F1F033F7200065
:1003E0001302120093022000E31E52FCB70E0F000E
:1003F000938EFE00930110016310D71D13020000BD
:1004000037110F0F1301F1F0B70001FF938000F0D7
:1004100033F720001302120093022000E31252FE71
:10042000B71E000F938E0EF0930120016316D719AB
:100430001302000037F1F0F01301010FB710F00FB5
:10044000938000FF1300000033F720001302120016
:1004500093022000E31052FEB70EF000938E0E0FB1
:1004600093013001631AD7151302000037110F0FE3
:100470001301F1F0B700FF009380F00F13000000AC
:100480001300000033F72000130212009302200033
:10049000E31E52FCB70E0F00938EFE009301400145
:1004A000631CD7111302000037110F0F1301F1F075
:1004B00013000000B70001FF938000F033F7200025
:1004C0001302120093022000E31052FEB71E000F29
:1004D000938E0EF0930150016310D70F13020000AA
:1004E00037F1F0F01301010F13000000B710F00F07
:1004F000938000FF1300000033F720001302120066
:1005000093022000E31E52FCB70EF000938E0E0FF4
:10051000930160016312D70B1302000037110F0F14
:100520001301F1F01300000013000000B700FF00FA
:100530009380F00F33F72000130212009302200083
:10054000E31E52FCB70E0F00938EFE009301700164
:100550006314D707B70001FF938000F033711000D8
:10056000930E0000930180016318D105B700FF00CE
:100570009380F00F33F10000930E0000930190017F
:10058000631CD103B3700000930E00009301A0011F
:100590006394D003B71011119380101137212222D8
:1005A0001301212233F02000930E00009301B001CB
:1005B0006314D001631030020F00F00F638001005C
:1005C0009391110093E111009308D0051385010068
:1005D000730000000F00F00F930110009308D00586
:1005E0001305000073000000731000C0000000003D
:0C05F000000000000000000000000000FF
:1010000000000000000000000000000000000000E0
:1010100000000000000000000000000000000000D0
:1010200000000000000000000000000000000000C0
:1010300000000000000000000000000000000000B0
:081040000000000000000000A8
:040000058000000077
:00000001FF
